:100000000C945D000C9485000C9485000C94850084
:100010000C9485000C9485000C9485000C9485004C
:100020000C9485000C9485000C9485000C9485003C
:100030000C9485000C9485000C9485000C9485002C
:100040000C94AD020C9485000C9474050C94A605D8
:100050000C9485000C9485000C9485000C9485000C
:100060000C9485000C94850000000008000201003B
:100070000003040700000000000000000102040863
:100080001020408001020408102001020408102002
:10009000040404040404040402020202020203032E
:1000A0000303030300000000250028002B000000CC
:1000B0000000240027002A00D60511241FBECFEF20
:1000C000D8E0DEBFCDBF11E0A0E0B1E0E0EDFDE0A3
:1000D00002C005900D92A831B107D9F721E0A8E13F
:1000E000B1E001C01D92A63EB207E1F710E0CAEBF5
:1000F000D0E004C02297FE010E94CC06C83BD10785
:10010000C9F70E9499060C94E6060C94000081E061
:1001100090E00E94D0069FEF980F923040F082E06E
:100120008093060162E081E090E00C94D806809311
:100130000601089526E040E855E260E070E089E4B9
:1001400091E00E94180543E050E060E070E089E42F
:1001500091E00E946F0661E086E00E94C60361E0C4
:1001600089E00E94C60361E087E00E94C60361E067
:1001700088E00E94C60360E070E086E00E943E03D3
:1001800060E070E089E00E943E03109239010C9417
:100190008700682F81E090E00C94D8060F931F939E
:1001A0000E94F70220910601223019F5E091180112
:1001B00024E0E29FF0011124E75EFE4F00811181EF
:1001C00022813381DC01CB01801B910BA20BB30B8D
:1001D000853F9140A105B10560F060E070E086E0E8
:1001E0000E943E0360E070E089E00E943E031092AE
:1001F00039011F910F91089589E491E00E9435041F
:10020000181619060CF0A7C144E050E06CE371E049
:1002100089E491E00E94750680913C0190913D0136
:1002200090933B0190913F0190933A01863609F4F7
:1002300049C1B8F5833409F487C040F4813409F426
:100240007DC0823409F087C182E079C0843609F428
:1002500014C1853609F07FC160E070E086E00E943D
:100260003E0360E070E089E00E943E0360E088E0C9
:100270000E94FF0360913B0170E089E00E943E0311
:1002800086E08093180180E4809339010E94F70290
:100290006093310170933201809333019093340164
:1002A0005AC1893609F4BAC0A8F5873609F42FC1B6
:1002B000883609F050C160E070E086E00E943E039D
:1002C00060E070E089E00E943E0360E087E00E9409
:1002D000FF0360913B0170E086E00E943E0360E016
:1002E00088E00E94FF0360913A0170E089E00E947B
:1002F0003E0381E08093180182E0809339010E94DF
:10030000F70260931D0170931E0180931F0190936B
:10031000200121C18B3609F452C018F18C3609F046
:100320001AC160E070E086E00E943E0360E070E089
:1003300089E00E943E03109239010DC181E0809353
:1003400006010E94C90007C16091060189E491E09D
:100350000E94B3046091390189E491E00E94B304E2
:10036000FAC060E070E086E00E943E0360E070E06A
:1003700089E00E943E0361E087E00E94FF036091F4
:100380003B0170E086E00E943E0360E088E00E944E
:10039000FF0360913A0170E089E00E943E031092F1
:1003A000180181E0809339010E94F70260931901DE
:1003B00070931A0180931B0190931C01CCC060E0E4
:1003C00070E086E00E943E0360E070E089E00E94F9
:1003D0003E0360E087E00E94FF0360913B0170E014
:1003E00086E00E943E0361E088E00E94FF03609186
:1003F0003A0170E089E00E943E0382E08093180198
:1004000084E0809339010E94F70260932101709388
:10041000220180932301909324019DC060E070E04D
:1004200086E00E943E0360E070E089E00E943E03A7
:1004300061E087E00E94FF0360913B0170E086E08D
:100440000E943E0361E088E00E94FF0360913A0150
:1004500070E089E00E943E0383E08093180188E009
:10046000809339010E94F702609325017093260161
:1004700080932701909328016EC060E070E086E0D1
:100480000E943E0360E070E089E00E943E0360E06D
:1004900087E00E94FF0360913B0170E086E00E94CC
:1004A0003E0384E08093180180E1809339010E942B
:1004B000F7026093290170932A0180932B01909396
:1004C0002C0149C060E070E086E00E943E0360E0DD
:1004D00070E089E00E943E0361E087E00E94FF0334
:1004E00060913B0170E086E00E943E0385E08093CE
:1004F000180180E2809339010E94F70260932D0178
:1005000070932E0180932F019093300124C060E0FE
:1005100070E086E00E943E0360E070E089E00E94A7
:100520003E0361E088E00E94FF0360913B0170E0C0
:1005300089E00E943E0387E08093180180E8809361
:1005400039010E94F7026093350170933601809360
:100550003701909338010C94CE001F920F920FB682
:100560000F9211242F933F938F939F93AF93BF9339
:100570008091410190914201A0914301B0914401C9
:100580003091400126E0230F2D3720F40296A11D63
:10059000B11D05C029E8230F0396A11DB11D2093AD
:1005A00040018093410190934201A0934301B09395
:1005B00044018091450190914601A0914701B0917D
:1005C00048010196A11DB11D8093450190934601FC
:1005D000A0934701B0934801BF91AF919F918F9134
:1005E0003F912F910F900FBE0F901F9018952FB72E
:1005F000F894609141017091420180914301909182
:1006000044012FBF0895789484B5826084BD84B579
:10061000816084BD85B5826085BD85B5816085BDFD
:10062000EEE6F0E0808181608083E1E8F0E0108216
:10063000808182608083808181608083E0E8F0E057
:10064000808181608083E1EBF0E080818460808341
:10065000E0EBF0E0808181608083EAE7F0E0808178
:100660008460808380818260808380818E7F8083AC
:100670008081806880831092C10008951F93CF937A
:10068000DF93182FEB0161E00E94C603209711F45D
:1006900060E004C0CF3FD10539F461E0812FDF91E4
:1006A000CF911F910C94FF03E12FF0E0E859FF4F29
:1006B000E491E330F9F048F4E130B9F0E230A1F52B
:1006C00084B5806284BDC8BD34C0E730E9F0E8304D
:1006D00019F1E43049F580918000806280938000B8
:1006E000D0938B00C0938A0024C084B5806884BDF9
:1006F000C7BD1FC080918000806880938000D09328
:100700008900C093880015C08091B00080688093F4
:10071000B000C093B3000DC08091B00080628093A0
:10072000B000C093B40005C0C038D1050CF0B5CFFF
:10073000AFCFDF91CF911F910895833081F028F4DE
:10074000813099F08230A1F008958730A9F0883087
:10075000B9F08430D1F4809180008F7D03C0809106
:1007600080008F7780938000089584B58F7702C0D2
:1007700084B58F7D84BD08958091B0008F7703C0CC
:100780008091B0008F7D8093B0000895CF93DF9368
:1007900090E0FC01E458FF4F2491FC01E057FF4F2B
:1007A0008491882349F190E0880F991FFC01E2555C
:1007B000FF4FA591B4918C559F4FFC01C591D491E9
:1007C0009FB7611108C0F8948C91209582238C9377
:1007D000888182230AC0623051F4F8948C91322FC0
:1007E000309583238C938881822B888304C0F8946E
:1007F0008C91822B8C939FBFDF91CF9108950F93A3
:100800001F93CF93DF931F92CDB7DEB7282F30E031
:10081000F901E859FF4F8491F901E458FF4F149111
:10082000F901E057FF4F04910023C9F0882321F01C
:1008300069830E949D036981E02FF0E0EE0FFF1FA6
:10084000EC55FF4FA591B4919FB7F8948C9161112D
:1008500003C01095812301C0812B8C939FBF0F9003
:10086000DF91CF911F910F910895FC01818D228D11
:1008700090E0805C9F4F821B91098F7399270895A8
:10088000FC01918D828D981731F0828DE80FF11D5A
:10089000858D90E008958FEF9FEF0895FC01918D75
:1008A000828D981761F0828DDF01A80FB11D5D96D2
:1008B0008C91928D9F5F9F73928F90E008958FEF40
:1008C0009FEF08958CEC95E0892B49F080E090E053
:1008D000892B29F00E94CC0581110C940000089509
:1008E000FC01848DDF01A80FB11DA35ABF4F2C91CD
:1008F000848D90E001968F739927848FA689B7899C
:100900002C93A089B1898C9180648C93938D848D74
:10091000981306C00288F389E02D80818F7D808343
:100920000895CF93DF93EC01888D8823C9F0EA897D
:10093000FB89808185FD05C0A889B9898C9186FDD8
:100940000FC00FB607FCF5CF808185FFF2CFA889D5
:10095000B9898C9185FFEDCFCE010E947004E7CF5D
:10096000DF91CF910895CF92DF92FF920F931F9363
:10097000CF93DF931F92CDB7DEB76C0181E0D60134
:1009800058968C9358975B969C915B975C968C914C
:100990005C97981307C05096ED91FC915197808118
:1009A00085FD2EC0F601038D10E00F5F1F4F0F7302
:1009B0001127F02EF601848DF81211C00FB607FC36
:1009C000F9CFD6015096ED91FC915197808185FF2A
:1009D000F1CFC60169830E9470046981EBCF838DDA
:1009E000E80FF11DE35AFF4F6083D6015B960C932D
:1009F0005B975296ED91FC915397808180620CC079
:100A0000D6015696ED91FC91579760835096ED91E3
:100A1000FC91519780818064808381E090E00F9009
:100A2000DF91CF911F910F91FF90DF90CF900895AC
:100A3000BF92CF92DF92EF92FF92CF93DF93EC01C0
:100A40006A017B01B22E60E874E88EE190E0A701B4
:100A500096010E94A8062150310941095109569575
:100A6000479537952795E889F98982E08083211594
:100A700080E1380798F0E889F989108260E472E42F
:100A80008FE090E0A70196010E94A806215031094D
:100A9000410951095695479537952795EC85FD8570
:100AA0003083EE85FF852083188EEC89FD89B08226
:100AB000EA89FB89808180618083EA89FB89808162
:100AC00088608083EA89FB89808180688083EA89E5
:100AD000FB8980818F7D8083DF91CF91FF90EF90A4
:100AE000DF90CF90BF9008951F920F920FB60F9294
:100AF00011242F938F939F93EF93FF93E0915901CC
:100B0000F0915A018081E0915F01F091600182FDD6
:100B100012C09081809162018F5F8F732091630179
:100B2000821751F0E0916201F0E0E75BFE4F958F94
:100B30008093620101C08081FF91EF919F918F911D
:100B40002F910F900FBE0F901F9018951F920F922C
:100B50000FB60F9211242F933F934F935F936F9390
:100B60007F938F939F93AF93BF93EF93FF9389E40A
:100B700091E00E947004FF91EF91BF91AF919F911E
:100B80008F917F916F915F914F913F912F910F9036
:100B90000FBE0F901F90189589E491E00E943504D4
:100BA00021E0892B09F420E0822F089510924C0156
:100BB00010924B0188EE93E0A0E0B0E080934D01ED
:100BC00090934E01A0934F01B09350018BE091E0C0
:100BD00090934A018093490185EC90E090935601EF
:100BE0008093550184EC90E09093580180935701D5
:100BF00080EC90E090935A018093590181EC90E051
:100C000090935C0180935B0182EC90E090935E0195
:100C100080935D0186EC90E09093600180935F018A
:100C200010926201109263011092640110926501AA
:100C30000895CF92DF92EF92FF920F931F93CF937D
:100C4000DF937C016A01EB0100E010E00C151D054B
:100C500071F06991D701ED91FC910190F081E02D47
:100C6000C7010995892B19F00F5F1F4FEFCFC801FE
:100C7000DF91CF911F910F91FF90EF90DF90CF9078
:100C800008950F931F93CF93DF93EC010E94F70217
:100C9000688779878A879B87E881F9810680F78151
:100CA000E02DCE01099597FF15C00E94F702088537
:100CB00019852A853B85601B710B820B930B0C8178
:100CC0001D812E813F81601771078207930720F3F2
:100CD0008FEF9FEFDF91CF911F910F910895FC014E
:100CE00044835583668377830895CF92DF92EF9292
:100CF000FF920F931F93CF93DF937C016A01EB0167
:100D000000E010E00C151D0549F0C7010E944106E6
:100D100097FD04C089930F5F1F4FF4CFC801DF9187
:100D2000CF911F910F91FF90EF90DF90CF9008959A
:100D300008950E9403030E9498060E949A00C2E64A
:100D4000D4E00E94FC002097E1F30E946204F9CFF6
:100D5000A1E21A2EAA1BBB1BFD010DC0AA1FBB1FBF
:100D6000EE1FFF1FA217B307E407F50720F0A21B31
:100D7000B30BE40BF50B661F771F881F991F1A949E
:100D800069F760957095809590959B01AC01BD01C8
:100D9000CF010895EE0FFF1F0590F491E02D099407
:100DA000F999FECF92BD81BDF89A992780B5089533
:100DB000262FF999FECF1FBA92BD81BD20BD0FB677
:100DC000F894FA9AF99A0FBE01960895F894FFCF15
:100DD0000000E60180000200000000B3041906359F
:080DE000044E044004910400DC
:107800000C94343C0C94513C0C94513C0C94513CE1
:107810000C94513C0C94513C0C94513C0C94513CB4
:107820000C94513C0C94513C0C94513C0C94513CA4
:107830000C94513C0C94513C0C94513C0C94513C94
:107840000C94513C0C94513C0C94513C0C94513C84
:107850000C94513C0C94513C0C94513C0C94513C74
:107860000C94513C0C94513C11241FBECFEFD8E036
:10787000DEBFCDBF11E0A0E0B1E0EAE8FFE702C063
:1078800005900D92A230B107D9F712E0A2E0B1E065
:1078900001C01D92AD30B107E1F70E942D3D0C945F
:1078A000C33F0C94003C982F95959595959595958B
:1078B000905D8F708A307CF0282F295A8091C0000B
:1078C00085FFFCCF9093C6008091C00085FFFCCF60
:1078D0002093C6000895282F205DF0CF982F809127
:1078E000C00085FFFCCF9093C6000895EF92FF92F1
:1078F0000F931F93EE24FF2487018091C00087FD22
:1079000017C00894E11CF11C011D111D81E2E8164D
:1079100081EAF80687E0080780E0180770F3E09135
:107920000401F091050109958091C00087FFE9CF1E
:107930008091C6001F910F91FF90EF9008950E94D3
:10794000763C982F8091C00085FFFCCF9093C600B5
:1079500091362CF490330CF09053892F089597555D
:10796000892F08951F930E949F3C182F0E949F3CCF
:107970001295107F810F1F9108951F93182F882350
:1079800021F00E94763C1150E1F71F9108951F935A
:10799000182F0E94763C803249F0809103018F5F5E
:1079A000809303018530C1F01F9108958091C0003C
:1079B00085FFFCCF84E18093C6008091C00085FFE5
:1079C000FCCF1093C6008091C00085FFFCCF80E102
:1079D0008093C6001F910895E0910401F091050184
:1079E00009951F9108950E94763C803241F0809164
:1079F00003018F5F80930301853081F008958091AA
:107A0000C00085FFFCCF84E18093C6008091C00058
:107A100085FFFCCF80E18093C6000895E0910401CA
:107A2000F09105010995089548EC50E08823A1F0F4
:107A30002D9A28EE33E0FA013197F1F721503040CA
:107A4000D1F72D9828EE33E0FA013197F1F7215064
:107A50003040D1F7815061F708953F924F925F9285
:107A60006F927F928F929F92AF92BF92CF92DF924E
:107A7000EF92FF920F931F93CF93DF93000082E06A
:107A80008093C00080E18093C4001092C50088E11B
:107A90008093C10086E08093C2005098589A259A3E
:107AA00081E00E94143D24E1F22E9EE1E92E85E959
:107AB000D82E0FE0C02E10E1B12EAA24A394B1E479
:107AC0009B2EA6E58A2EF2E57F2EE0E26E2E79E46B
:107AD000572E63E5462E50E5352E0E94763C8033C6
:107AE000B1F18133B9F1803409F46FC0813409F404
:107AF00076C0823409F485C0853409F488C08035A5
:107B000031F1823521F1813511F1853509F485C0D6
:107B1000863509F48DC0843609F496C0843709F49B
:107B200003C1853709F472C1863709F466C08091B4
:107B300003018F5F80930301853079F6E0910401A2
:107B4000F091050109950E94763C803351F60E9420
:107B5000F33CC3CF0E94763C803249F78091C0004D
:107B600085FFFCCFF092C6008091C00085FFFCCF5E
:107B70009092C6008091C00085FFFCCF8092C60025
:107B80008091C00085FFFCCF7092C6008091C0003C
:107B900085FFFCCF6092C6008091C00085FFFCCFBE
:107BA0005092C6008091C00085FFFCCF4092C60075
:107BB0008091C00085FFFCCF3092C6008091C0004C
:107BC00085FFFCCFB092C60088CF0E94763C8638F5
:107BD00008F4BDCF0E94763C0E94F33C7ECF0E9409
:107BE000763C803809F49CC0813809F40BC1823896
:107BF00009F430C1883909F48FC080E00E94C73C85
:107C00006CCF84E10E94BD3C0E94F33C66CF85E0CE
:107C10000E94BD3C0E94F33C60CF0E94763C809362
:107C200006010E94763C809307010E94F33C55CFE9
:107C30000E94763C803309F411C183E00E94BD3C70
:107C400080E00E94C73C49CF0E94763C80930902A5
:107C50000E94763C8093080280910C028E7F809374
:107C60000C020E94763C853409F409C18091080217
:107C700090910902892B89F000E010E00E94763C87
:107C8000F801E85FFE4F80830F5F1F4F809108026D
:107C9000909109020817190788F30E94763C8032F8
:107CA00009F045CF80910C0280FFF5C0609106017C
:107CB00070910701660F771F7093070160930601AB
:107CC000A0910802B09109021097C9F0E8E0F1E034
:107CD0009B01AD014E0F5F1FF999FECF32BD21BD53
:107CE000819180BDFA9AF99A2F5F3F4FE417F5070B
:107CF00099F76A0F7B1F70930701609306018091CB
:107D0000C00085FFFCCFF092C6008091C00085FFC7
:107D1000FCCFB092C600E1CE83E00E94C73CDDCE2E
:107D200082E00E94C73CD9CE0E94763C8093090233
:107D30000E94763C80930802809106019091070191
:107D4000880F991F90930701809306010E94763C4B
:107D5000853409F49AC080910C028E7F80930C02C6
:107D60000E94763C803209F0B8CE8091C00085FF39
:107D7000FCCFF092C600A0910802B09109021097C2
:107D8000C1F180910C02082F0170182F1695117007
:107D9000E0910601F0910701AF014F5F5F4FBA011B
:107DA00020E030E00023B1F4112339F49491809164
:107DB000C00085FFFCCF9093C6002F5F3F4FCB01E3
:107DC0000196FA012A173B0780F4BC014F5F5F4F11
:107DD000002351F3F999FECFF2BDE1BDF89A90B5B9
:107DE0008091C00085FFFCCFE6CF709307016093C0
:107DF00006018091C00085FDE5CE8091C00085FF21
:107E0000F8CFE0CE81E00E94C73C67CE0E94763C6E
:107E1000803209F08CCE8091C00085FFFCCFF092BB
:107E2000C6008091C00085FFFCCFE092C600809123
:107E3000C00085FFFCCFD092C6008091C00085FFB6
:107E4000FCCFC092C6008091C00085FFFCCFB092ED
:107E5000C60043CE80E10E94C73C3FCE0E94763CE4
:107E60000E94763C182F0E94763C112309F483C0AF
:107E7000113009F484C08FE00E94C73C2ECE80915F
:107E80000C02816080930C02F1CE80910C02816023
:107E900080930C0265CF809107018823880F880B9F
:107EA0008A2180930B028091060190910701880F2F
:107EB000991F90930701809306018091080280FF2B
:107EC00009C08091080290910902019690930902DD
:107ED00080930802F894F999FECF1127E0910601EA
:107EE000F0910701C8E0D1E0809108029091090269
:107EF000103091F40091570001700130D9F303E084
:107F000000935700E8950091570001700130D9F3B4
:107F100001E100935700E8950990199000915700EE
:107F200001700130D9F301E000935700E8951395F3
:107F3000103498F011270091570001700130D9F3E7
:107F400005E000935700E89500915700017001305B
:107F5000D9F301E100935700E8953296029709F0B2
:107F6000C7CF103011F00296E5CF11248091C000E8
:107F700085FFC5CEC8CE8EE10E94C73CAECD85E957
:0A7F80000E94C73CAACDF894FFCF81
:027F8A00800075
:040000030000780081
:00000001FF
